:020000006B286B
:1000080064000C1E0428990003146628A301A200AA
:10001800FF30A207031CA307031C66280330A100B6
:10002800E43018200C28A101F63EA000A109031C09
:100038002328FE300000A00703181E28A00764002C
:10004800A10F1D2800002018292820182B28080097
:100058000310A10CA00CFF3E03182C2820086628CA
:10006800A501A4011030A600210DA40DA50D22089C
:10007800A4022308031C230FA50203184A282208F8
:10008800A40723080318230FA5070310A00DA10D2B
:10009800A60B3828200866281030A800A101A00166
:1000A800A70CA60C031C5E282208A0072308031827
:1000B800230FA107A10CA00CA50CA40CA80B542875
:1000C8002408662883130313831264000800831628
:1000D80007309900203098008312903098008316DA
:1000E80007309F0081178312861183168611071027
:1000F80087100711071287128312B030DE00103004
:10010800C100C0014030C7008316860183128716DC
:10011800831687128312871083168710831287101D
:1001280083168710C83083128A010A208714831621
:1001380087108312871483168710831287128316F9
:100148008712533083128A01042074308A010420F4
:1001580061308A01042072308A01042074308A01D7
:10016800042069308A0104206E308A010420673037
:100178008A0104202E308A0104202E308A010420AE
:100188002E308A0104200D308A0104200A308A01A9
:1001980004208A110A122E2A8710831687103230FB
:1001A80083128A0117208714831687108312E2307E
:1001B800CC008A110A120921A230CC008A110A1235
:1001C8000921A030CC008A110A120921C830CC00BC
:1001D8008A110A1209212630CC008A110A12092133
:1001E8008130CC008A110A1209212030CC008A11F2
:1001F8000A1209212F30CC008A110A120921AF30C6
:10020800CC008A110A120921080007168316071262
:100218008312071183160711831287128316871218
:10022800831207108316071083124C0886000714E0
:100238008316071083128716831687128312080005
:1002480007168316071283120715831607118312E0
:1002580087128316871283120710831607108312DA
:100268005008860007148316071083128716831612
:100278008712831208008316FF3086008312071442
:10028800831607108312071183160711831287122A
:100298008316871283120712831607128312060821
:1002A800D300071683160712831287168316871240
:1002B800860183120800B030DE006400B8305E02A8
:1002C8008A110A1203188D294030CC008A010921AD
:1002D8005E08CC008A0109211030CC008A0109216E
:1002E8000430CC008A0109210430C3006400843042
:1002F80043028A110A12031888298A012421C30A91
:100308008A110A12031D7A29DE0A8A110A12031DAC
:1003180061290800D0018A015F2108004030CC0023
:100328008A0109215708A000A1010830A200A301F1
:100338008A013420B2002108B300B0303207DF0050
:100348005F08CC008A01092104305407DA005A08F2
:10035800A000A10104308A012F20B2002108B300B7
:1003680010303204CC008A0109210F305A05CC0024
:100378008A0109214B08D0008A0124210800203075
:100388003E02BD00640050303E028A110A12031C6E
:10039800D02950303E02BD003D08A600A701053017
:1003A800A200A3018A015020C5000130C8006400E2
:1003B800063048028A110A120318FC2964005030DA
:1003C8003E028A110A12031CF0298A110A12F22429
:1003D800C50A8A110A12F4298A110A12D523C50AF4
:1003E8008A019221D40AC80A8A110A12031DDB293C
:1003F800D40ACB018A01922108005708A000A10164
:100408000830A200A3018A013420B2002108B300F9
:10041800B0303207DF005F08CC008A010921403084
:10042800CC008A01092104305407DA005A08A000D8
:10043800A10104308A012F20B2002108B300103036
:100448003204CC008A0109210F305A05CC008A01F8
:10045800092108004C308A01042043308A01042015
:1004680044308A01042020308A01042069308A013E
:1004780004206E308A01042069308A010420743017
:100488008A0104202E308A0104202E308A0104209B
:100498002E308A0104200D308A0104200A308A0196
:1004A80004208A01D0208A018E210830D70010301C
:1004B800D400E2016400123062028A110A120318A1
:1004C8008F2A6208113C8A110A12031C882A8A1191
:1004D8000A127222BE008A110A12882A02308A0081
:1004E800620882074F347034743472346534783457
:1004F800203446342D3435343134333432343034C6
:1005080020344C34433444348A01C321E20A8A112A
:100518000A12031D5E2A1030D7002430D400E201ED
:1005280064000B3062028A110A120318BE2A62089C
:100538000A3C8A110A12031CB72A8A110A12A82235
:10054800BE008A110A12B72A02308A00620882079E
:100558004734723461347034683469346334203415
:100568004C34433444348A01C321E20A8A110A1202
:10057800031D942A1030D7000830D400E20164002B
:10058800083062028A110A120318EB2A6208073C33
:100598008A110A12031CE32A8A110A12D722CB00F5
:1005A8008A110A12E32A02308A0062088207C334D9
:1005B800A534993481349934A534C3340034D40A29
:1005C8008A019221E20A8A110A12031DC32A1030F5
:1005D800D7001430D400E2016400083062028A11A6
:1005E8000A120318182B6208073C8A110A12031C06
:1005F800102B8A110A120423CB008A110A12102B1D
:1006080003308A0062088207183418341834183402
:100618007E34423424341834D40A8A019221E20AFE
:100628008A110A12031DF02A1030D7006730D4004F
:10063800E2016400083062028A110A120318452B8D
:100648006208073C8A110A12031C3D2B8A110A1200
:100658003123CB008A110A123D2B03308A0062082D
:1006680082072634463480349034903480344634BB
:100678002634D40A8A019221E20A8A110A12031D39
:100688001D2B1030D7007130D400E201640008300F
:1006980062028A110A120318722B6208073C8A1137
:1006A8000A12031C6A2B8A110A125E23CB008A11D4
:1006B8000A126A2B03308A0062088207FF348134E9
:1006C800BD34A534A534BD348134FF34D40A8A013D
:1006D8009221E20A8A110A12031D4A2B2030D70000
:1006E8003C30D400E2016400083062028A110A1228
:1006F80003189F2B6208073C8A110A12031C972BC8
:100708008A110A128B23CB008A110A12972B033005
:100718008A0062088207603460341F340334C634A8
:10072800FC3400340034D40A8A019221E20A8A1186
:100738000A12031D772B3030D7001830D400E2019D
:1007480064000F3062028A110A120318D22B620861
:100758000E3C8A110A12031CCB2B8A110A12B823E9
:10076800BE008A110A12CB2B03308A006208820766
:1007780028346334293443344F344D34503453349B
:1007880079347334203432343034303435348A0197
:10079800C321E20A8A110A12031DA42B64008A01EC
:1007A800D22B4508EF3C8A110A12031CF12C8A113E
:1007B8000A12E223CB008A110A12F12C04308A00B3
:0407C8004508002CB4
:1008000082070034003400340034003400340034F3
:100810005F340034003400340734003407340034CB
:1008200014347F3414347F34143424342A347F3421
:100830002A341234233413340834643462343634A2
:1008400049345534223450340034053403340034F0
:10085000003400341C342234413400340034413438
:1008600022341C340034143408343E340834143434
:10087000083408343E3408340834003450343034FA
:1008800000340034083408340834083408340034A0
:1008900060346034003400342034103408340434BC
:1008A00002343E345134493445343E340034423409
:1008B0007F34403400344234613451344934463456
:1008C0002134413445344B34313418341434123427
:1008D0007F341034273445344534453439343C347E
:1008E0004A344934493430340134713409340534DC
:1008F00003343634493449344934363406344934BF
:10090000493429341E34003436343634003400344B
:10091000003456343634003400340834143422346D
:100920004134003414341434143414341434003482
:10093000413422341434083402340134513409343B
:10094000063432344934793441343E347E341134FF
:10095000113411347E347F344934493449343634C7
:100960003E3441344134413422347F3441344134C3
:1009700022341C347F3449344934493441347F347F
:1009800009340934093401343E344134493449349A
:100990007A347F340834083408347F3400344134E6
:1009A0007F34413400342034403441343F34013406
:1009B0007F3408341434223441347F34403440349A
:1009C000403440347F3402340C3402347F347F347A
:1009D0000434083410347F343E34413441344134DB
:1009E0003E3408004508EF3C8A110A12031CF32D1F
:1009F0008A110A12FF24CB008A110A12F32D053046
:100A00008A00450882077F340934093409340634E2
:100A10003E344134513421345E347F340934193446
:100A20002934463446344934493449343134013464
:100A300001347F34013401343F3440344034403495
:100A40003F341F342034403420341F343F3440348A
:100A5000383440343F346334143408341434633449
:100A6000073408347034083407346134513449345D
:100A70004534433400347F3441344134003402344B
:100A800004340834103420340034413441347F3489
:100A90000034043402340134023404344034403429
:100AA00040344034403400340134023404340034DF
:100AB000203454345434543478347F3448344434F7
:100AC00044343834383444344434443420343834AE
:100AD0004434443448347F343834543454345434F3
:100AE000183408347E340934013402340C3452345E
:100AF000523452343E347F3408340434043478346D
:100B0000003444347D3440340034203440344434A0
:100B10003D3400347F3410342834443400340034FD
:100B200041347F34403400347C3404341834043489
:100B300078347C340834043404347834383444341D
:100B40004434443438347C34143414341434083485
:100B500008341434143418347C347C3408340434A9
:100B60000434083448345434543454342034043471
:100B70003F344434403420343C3440344034203416
:100B80007C341C342034403420341C343C34403415
:100B9000303440343C344434283410342834443421
:100BA0000C345034503450343C3444346434543471
:100BB0004C34443400340834363441340034003486
:100BC00000347F3400340034003441343634083487
:100BD000003410340834083410340834783446347F
:0E0BE000413446347834080063008A01F42D55
:02400E003D3D36
:00000001FF
